:030000000203B147
:03004300020100B7
:1001000002013C000201580002011800020129000E
:10011000020120000201180032E591C2E4F59122AB
:10012000C0E0C2003119D0E032C0E0E5874401F5FB
:10013000870000003119D0E032C2DC32C0D0C0E00C
:10014000C082C08312016931197401907FABF0D075
:1001500083D082D0E0D0D032C0D0C0E0C082C08393
:090160001204283119740280E236
:10016900907FE8E0A2E79202545C7051E0A2E0823D
:10017900E1404A30E50274035403C4F540A3E05456
:100189000F45401201D52001343002182003209078
:100199007F027846754003E6F0158218D540F8E6E7
:1001A900907FB5F0754002907FB4E04540F022851C
:1001B9008240E583907FD4F0E540A380E675400353
:1001C90080E5E02582F58250020583229001FA310B
:1001D900CCE09001FA31CCC082C0837845E4F618AE
:1001E900F6187601907FEAE0F5F0A3E0C201C203B8
:1001F900226D404040404081406A74404040404048
:1002090040714040404040A540404040404040404F
:1002190040714240404040404040404040404040A2
:1002290040405663404040404040435D404040406C
:1002390040D201223000FA907FC5F0907FAAE054A5
:100249000160FBF00204163000E70876182230003E
:10025900E0F541223000DA08A641223000D50876BF
:100269000122760222E5F060061470C5D20022C28E
:100279000022D203149002C560B9149002D760B36A
:100289001470AE900315E5F0601EF54031CBE060C7
:10029900A0E5401480F2D203C394219002E960934F
:1002A900149002F9608D8089E0FFF5F07800F2087A
:0C02B900A3E0DFFAD0E0D0E0E5F021A9DE
:1002C500120101010000004042420001000101024B
:1002D5000001090222000101038032090400000126
:1002E50003000004092100010001221C000705810B
:1002F500034000640600FF0901A101190129081541
:10030500002501750195088102190129089102C08E
:10031500040309042C035500530042002000440047
:1003250065007300690067006E00200042007900D7
:1003350020004500780061006D0070006C006500CC
:10034500220342007500740074006F006E00730094
:100355002000260020004C0069006700680074003A
:1003650073002403530069006D0070006C00650084
:10037500200049002F004F00200044006500760052
:10038500690063006500240346006900720073007C
:100395007400200048004900440020004500780012
:1003A50061006D0070006C00650000007581EB75E3
:1003B500927F78D6E254F3F2120405E24406F2E4A1
:1003C500F520F548F54604F547F542F5497893E4F7
:1003D500F2799CF4F30809E2540FF2E344F0F308D0
:1003E50009E254F0F2E3440FF3E478ACF208F208C2
:1003F5007403F2087401F275E80175A8C00080FD68
:1004050075406490FB50A3E582458370F9D540F3B0
:1004150022907EC0E0F54822907E80F0907FB774F0
:1004250001F022D54926754904E54723F547554886
:1004350012044C12043D80E0907F9AE054F0F540A0
:0D044500A3E0540F454022F4907F96F02272
:00000001FF
